:0C0F200002250000024900000221000030
:100E4B00E4FDFCC3ED9FEC9E5015E4FBFA0BBB00DD
:0F0E5B00010AEB64794A70F50DBD00010C80E4CB
:010E6A002265
:100F7200000000000000000000000000000000006F
:010F8200224C
:0E0F83007F307E02EF1FAC0670011E4C70F630
:010F9100223D
:0F0F9200D290D291120F72C290120F72C291229E
:0C100200C290D291120F72D290020F72B5
:0E0FB000A20092A0D2A1120F72C2A1020F7273
:0D0FE800D2A1120F72A2A0C2A1120F72229C
:100EA700E4FEEF25E0FF92A0D2A1120F72C2A112B9
:090EB7000F720EBE08EC020FE8F8
:100E6B00E4FFD2A0FEEF25E0FFD2A1120F72A2A0E9
:0D0E7B00E4334207C2A1120F720EBE08E858
:010E88002247
:100F6000AD07120F927F46120EA7AF05120EA70211
:020F700010026D
:100D9400120F927F47120EA7E4FD120E6B74412DC1
:100DA400F8A607BD0304D2008002C200120FB00DE2
:090DB400BD03E7121002020F83D7
:051033007F01020F60C7
:100F0A00758921759850758DFD858D8BE4F587D28D
:060F1A00AFD2ACD28E2222
:07102C00AE071FEE70FA226F
:0E0FBE00C2ACC2998F993099FDC299D2AC2273
:100EF2001203D9FF6011120FBE7F0512102C74016C
:080F020029F9E43AFA80E92222
:10048B00E4F514F5157F01120F607F10120F607FDA
:10049B00B47E00120E4B120D94752300854124E59A
:1004AB0024FE7C00E42542F524EC3EF523FCAD2430
:1004BB0012031F7B9A7A997999783F1202048F3233
:1004CB008E318D308C2F120BA28E338F347C007DAE
:1004DB00641204478E338F34209252120FF5209200
:1004EB002AE52C452B7024E52A45297007F529753B
:1004FB002A018005E4F529F52AE52A6401452970CE
:10050B0006D2A3C2978004C2A3D297C3E515943237
:10051B00E51464809480501020920D120FF5051590
:10052B00E51570E7051480E3E4F514F515209364E5
:10053B00120FF520933CE52A4529601A054AE54A36
:10054B0070020549C39405E54964809480401EE41C
:10055B00F549F54A8017E52C452B7007F52B752CC3
:10056B00018005E4F52BF52CE4F525F5267F01122A
:10057B00100EC3E5159432E514648094805010205E
:10058B00930D120FF50515E51570E7051480E3E4DF
:10059B00F514F51520B741120FF520B7190528E50D
:1005AB002870020527D39463E52764809480400666
:1005BB00752700752863C3E5159432E514648094A0
:1005CB0080501020B70D120FF50515E51570E705D6
:1005DB001480E3E4F514F51520B63E120FF520B6A2
:1005EB0016E528152870021527C3E527648094802B
:1005FB005005E4F527F528C3E5159432E51464801E
:10060B009480501020B60D120FF50515E51570E707
:10061B00051480E3E4F514F51520A240120FF52024
:10062B00A2180526E52670020525C39404E525646A
:10063B008094804005E4F525F526C3E5159432E555
:10064B001464809480501020A20D120FF50515E54F
:10065B001570E7051480E3E4F514F51530A70302D4
:10066B00071C120FF530A70302071CE52645257062
:10067B001A0536E53670020535C39418E5356480E6
:10068B009480406BE4F535F5368064E526640145CE
:10069B0025701A0538E53870020537C3943BE537EA
:1006AB00648094804049E4F537F5388042E5266450
:1006BB00024525701A053CE53C7002053BC39418B6
:1006CB00E53B648094804027E4F53BF53C8020E5D6
:1006DB0026640345257018053EE53E7002053DC3B3
:1006EB00943BE53D648094804005E4F53DF53EC3C5
:1006FB00E5159432E51464809480501020A70D12F8
:10070B000FF50515E51570E7051480E3E4F514F511
:01071B0015C8
:01071C0022BA
:100A7D007D017C00E54DC4540F75F00AA4FFAEF066
:100A8D00E54D540F7A002FF515EA3EF514E54CC4EB
:100A9D00540F75F00AA4FFAEF0E54C540F2FF51767
:100AAD00EA3EF516C3E5159536E5356480F8E5148F
:100ABD00648098404BD3E515953CE53B6480F8E5A3
:100ACD001464809840028038E515B53618E514B5E4
:100ADD003513C3E5179538E5376480F8E51664805E
:100AED00985002801BE515B53C1AE514B53B15D39E
:100AFD00E517953EE53D6480F8E516648098400461
:080B0D00E4FEFF22AE04AF0577
:010B150022BD
:1009A000E52A45296003020A26120A7DEF4E60748B
:1009B000E4FFFE7DC87C42AB32AA31A930A82F12D9
:1009C00002A15060C3E528940AE527648094805012
:1009D0000EE5289400E5276480948040028055C38A
:1009E000E528940AE52764809480400EE528941455
:1009F000E527648094805002804CC3E5289414E578
:100A00002764809480400EE528941EE52764809436
:100A1000805002803FC3E528941EE52764809480BF
:100A2000404A803E8046E54A45496040E54A6401C7
:100A30004549700AC2A5C2A6C2A1D2A48036E54A21
:100A4000640245497006C2A5C2A6801AE54A64033D
:100A500045497006C2A5D2A6800CE54A6404454902
:100A60007012D2A5D2A6D2A1D2A48008C2A5C2A6D5
:0D0A7000C2A1C2A4E529452A24FF92A322B9
:100CFC00E4F508F509120F4C120F0A120EC07535E7
:100D0C0000753612E4F537F538F539F53AF53B75DB
:100D1C003C17F53D753E1EF53FF540120F36120798
:090D2C001D12048B1209A080F2D3
:10071D00E52C452B7F80600302089E12100EE54FDD
:10072D00C4540F2430FF121018E54F540F2430FF1E
:10073D001210187F2D121018E54EC4540F2430FFDF
:10074D00121018E54E540F2430FF1210187F20128E
:10075D001018E54DC4540F2430FF121018E54D54F8
:10076D000F2430FF1210187F3A121018E54CC454A4
:10077D000F2430FF121018E54C540F2430FF1210C7
:10078D00187F3A121018E54BC4540F2430FF121085
:10079D0018E54B540F2430FF1210187F201210183B
:1007AD00E550540F2430FF1210187FC012100EAFF9
:1007BD0032AE31AD30AC2F1203588E148F157C270D
:1007CD007D101203F28C148D15AE14AF157C037DC4
:1007DD00E81203F2EF2430FF121018AE14AF157C9F
:1007ED00037DE81203F28C148D15AE14AF157C0049
:1007FD007D641203F2EF2430FF121018AE14AF1502
:10080D007C007D641203F28C148D15AE14AF157C33
:10081D00007D0A1203F2EF2430FF121018AE14AF50
:10082D00157C007D0A1203F28C148D15E51524300C
:10083D00FF1210187F4C1210187F781210187F209D
:10084D00121018AE33AF347C007D0A120447EF242A
:10085D0030FF121018AE33AF347C007D0A120447FE
:10086D00ED2430FF1210187F431210187F20121044
:10087D0018AE27AF287C007D0A1204477C007D0A44
:10088D00120447ED2430FF121018AE27AF280209CD
:10089D009112100EAE35AF367C007D0A120447EF73
:1008AD002430FF121018AE35AF367C007D0A1204CD
:1008BD0047ED2430FF1210187F3A121018AE37AFE3
:1008CD00387C007D0A120447EF2430FF121018AE59
:1008DD0037AF387C007D0A120447ED2430FF12102B
:1008ED00187F3A121018AE39AF3A7C007D0A120407
:1008FD0047EF2430FF121018AE39AF3A7C007D0A55
:10090D00120447ED2430FF1210187F20121018E545
:10091D00262430FF1210187FC012100EAE3BAF3CD4
:10092D007C007D0A120447EF2430FF121018AE3BF5
:10093D00AF3C7C007D0A120447ED2430FF121018E5
:10094D007F3A121018AE3DAF3E7C007D0A1204476F
:10095D00EF2430FF121018AE3DAF3E7C007D0A1221
:10096D000447ED2430FF1210187F3A121018AE3FD5
:10097D00AF407C007D0A120447EF2430FF1210189F
:10098D00AE3FAF407C007D0A120447ED2430FF12CC
:02099D00101830
:01099F002235
:0C0FF5007F017E267D82DDFEDEFADFF645
:0110010022CC
:100D6A00C2958F807F017E00120D7BD2947F057E13
:010D7A000078
:100D7B00D3EF9400EE9400400F7DC77C01DCFEDDC9
:080D8B00FAEF1F70EB1E80E877
:010D9300223D
:0A100E00C294C296120D6AC2942229
:0A101800C294D296120D6AC294220F
:100EC0007F3812100E7F0C12100E7F0612100E7F4C
:090ED0000112100E7F8002100EC9
:0E0FCC0081838587898B8D80828486888A8CBC
:090F2C00074B0024120105072205
:100D3500C2B300C2B500D2B300E4FEEF1392B4EF24
:100D4500C313FFD2B500C2B5000EBE08EEE4FEED3A
:100D55001392B4EDC313FDD2B500C2B5000EBE08A3
:040D6500EEC2B30027
:010D69002267
:100BF100C2B300C2B500D2B300E4FDEF1392B4EF6B
:100C0100C313FFD2B500C2B5000DBD08EE00E4FD6F
:100C1100A2B4E433FFC43333335480FCEEC3134C2A
:100C2100FED2B500C2B5000DBD08E5C2B300D2B514
:090C310000C2B400D2B400AF0609
:010C3A002297
:100F4C00E4FD7F8E120D35E4FF0FBF07FC7D807F23
:040F5C008E020D35BF
:100F3600E4FBEB900FCC93FF120BF1744B2BF8A64E
:050F4600070BBB07EDE5
:010F4B002283
:050FDA00120FDFD2A19F
:080FDF007F017E02DEFEDFFA55
:010FE70022E7
:0F0FA100D2A0120FDAC2A0120FDFC2A1020FDF1F
:0A102200C2A0120FDAD2A0020FDF05
:020C7D00AD07C1
:100C7F00E4FBFAEDC4131313540124FF92A0ED25E6
:100C8F00E0FD120FDAC2A1120FDF0BBB08E5D2A0F5
:100C9F00120FDFD2A130A00F0AEAD394C840F6C2D8
:0E0CAF00A1120FDF7F0022C2A1120FDF7F0112
:010CBD002214
:100DBD00E4FDFCD2A0120FDFD2A1120FDFEC25E073
:100DCD00FCA2A0E4334204120FDFC2A1120FDF0D0B
:050DDD00BD08E5AF04B4
:010DE20022EE
:100ED900AC05A907120FA17FA0120C7DAF01120C5E
:090EE9007DAF04120C7D02102201
:020E0800AC0735
:100E0A00120FA17FA0120C7DAF04120C7D120FA14C
:0F0E1A007FA1120C7D120DBDAD07121022AF0586
:010E290022A6
:100E8900D3EF9400EE940040147D6E7C00ED1D704C
:0D0E9900011CED4C70F7EF1F70E61E80E3AA
:010EA6002229
:100DE300C2B27B46AF031BEF70FAD2B2E4FB30B260
:100DF300117F017E00120E890BEBD3940540EF7F28
:040E030000227F0149
:010E070022C8
:100CBE007D087C00C2B20FBF0000D2B20FBF000091
:100CCE000FBF0000A2B2E433C43333335480FBE9C8
:100CDE00C3134BF97E007F04EF1FAA0670011E4A54
:0D0CEE0070F6ED1D70011CED4C70C9AF01DA
:010CFB0022D6
:0C0C3B00120DE37F017E00120E897FCCB9
:100C4700E4FBFAC2B2051CE51C7002051BEF139208
:100C5700B2751B00751C06E51C151CAC1B70021534
:100C67001B4C70F3D2B2EFC313FF0BBB00010AEBAF
:050C770064084A70CE84
:010C7C002255
:100E2A00E4FFFE120C3B7F44120C47120C3B7FBEC0
:100E3A00120C47120CBE8F1A120CBEEFFEE51AFFF7
:010E4A002285
:100BA200120E2AC3EE9400500DEF1F70011E630750
:100BB200FF6306FF8000AD07AC06E412031FE4FBEF
:100BC200FA7980783D1200FB8F198E188D178C16DA
:100BD200E4FFFE7DC87C42AB19AA18A917A8161219
:0E0BE20000FBE4FBFAF9783F12000A120358F8
:010BF00022E2
:100003000203C4E86480F8E933E83360110460F064
:10001300ED33EC337009E8FCE9FDEAFEEBFF220463
:1000230060DED3EB9FEA9EE99DE8C2E78CF0C2F75E
:1000330095F0400CE8CCF8E9CDF9EACEFAEBCFFB2A
:1000430012038F85D0F05804700320D5B3E80470F1
:10005300075002B2D50203CE92D5EC0460F7E4CC8C
:10006300C0E0C398F8603B94186008400DD0E0FBF3
:100073000203A6E4FBFAC9FC8028E830E406E4C9DD
:10008300FBE4CAFCE830E305E4C9CACBFCE8540747
:100093006010F8C3E913F9EA13FAEB13FBEC13FC52
:1000A300D8F130F52FC3E49CFCEF9BFFEE9AFEEDF5
:1000B30099FDD0E0FBEF4E4D4C701222DB0302039F
:1000C300CBEC2CFCEF33FFEE33FEED33FDED30E7ED
:1000D300EB0203A6EF2BFFEE3AFEED39FDD0E0FB7A
:1000E30050130BBB00030203CEED13FDEE13FEEF23
:0800F30013FFEC13FC0203A64D
:1000FB00EC4D6011E8497017ED33EC3304600DE4FF
:10010B00FCFFFEFD22E933E8330470F80203C4124E
:10011B00038F58046009E4CC24815006285009024F
:10012B0003CE2840030203CBC0E0EB4A7044B980F6
:10013B0006D0E0FB0203BAEF4E701CBD8008EBFF4C
:10014B00EAFEE9FD80EBE98DF0A4FEE5F00201E4A7
:10015B00E9CDF9EAFEEBFFEF89F0A4FCE5F0CE89DF
:10016B00F0A42EFFE435F0CD89F0A42DFEE435F09C
:10017B008067EF4E7005BD80D780C3EF8BF0A4ACCA
:10018B00F0EE8BF0A42CFCE435F0F8EF8AF0A42C05
:10019B00E5F038FCE433CB8DF0A42CFCE5F03BF818
:1001AB00EE8AF0A42CFCE5F038F8E433CF89F0A408
:1001BB002CFCE5F038CF3400CE89F0A42FFFE5F00E
:1001CB003EFEE433C98DF0A42EFEE5F039CD8AF066
:1001DB00A42FFFE5F03EFEE43DFD33D0E0FB5007DE
:1001EB000BBB000F0203CEEC2CFCEF33FFEE33FE08
:0601FB00ED33FD0203A636
:100201000203CEEC5D046005E8590470030203C4E7
:1002110012038F580460F6EC4860F2EC7004FDFEA6
:10022100FF22C860DB2481C85009C39860025006D0
:100231000203CB9850CAF582E9294B4A7005AB827B
:100241000203BA75F0007C1A7880C3EF9BEE9AED39
:1002510099400DC3EF9BFFEE9AFEED99FDE842F048
:10026100DC23ACF0D0E0FFD0E0FED0E0FDAB82209B
:10027100E7101BEB60BAEC2CFCEF33FFEE33FEED25
:1002810033FD0203A6E803F830E705C0F075F0007E
:10029100EF2FFFEE33FEED33FD40B830E7C280AA09
:1002A10074F8CC6480CCC86480C8F58204604FC304
:1002B100EB9FF5F0EA9E42F0E99D42F0E89C45F0A3
:1002C100603C501DE5825FFFE582D313CB5BCBF42D
:1002D1002B5582FB50280ABA002409B90020088056
:1002E1001DE5825BFBE582D313CF5FCFF4C3132FF0
:1002F1005582FF50090EBE00050DBD00010CC3EB78
:100301009FF5F0EA9E42F0E99D42F0E89C45F060DD
:0903110007CC4820E701B3EC22FF
:10031A0075F020800E75F010800575F0087D007E5E
:10032A00007F003392D530D50312047DEC334010A0
:10033A00EF33FFEE33FEED33FDEC33FCD5F0ED2267
:0E034A00E5F0247EA2D513CC92E7CDCEFF22A3
:10035800EDD2E7CD33EC3392D524814006E4FFFE9D
:10036800FDFC22FCE4CFCECDCC24E0501174FF80FC
:10037800EDC3CC13CCCD13CDCE13CECF13CF047099
:07038800F030D5DE02047D18
:10038F00E9D2E7C933E833F892D5EDD2E7CD33ECB4
:07039F0033FC5002B2D5222D
:1003A600EC30E7100FBF000C0EBE00080DBD0004B8
:1003B6000BEB6014A2D5EB13FCED92E7FD2274FF64
:1003C600FCFDFEFF22E480F8A2D574FF13FC7D80BD
:0303D600E480EFD1
:03000000020B16DA
:0C0B1600787FE4F6D8FD758151020B5D7C
:1003D900BB010689828A83E0225002E722BBFE0222
:0903E900E32289828A83E4932255
:1003F200BC000BBE0029EF8DF084FFADF022E4CCEF
:10040200F875F008EF2FFFEE33FEEC33FCEE9DECB7
:10041200984005FCEE9DFE0FD5F0E9E4CEFD22EDFD
:10042200F8F5F0EE8420D21CFEADF075F008EF2F47
:10043200FFED33FD4007985006D5F0F222C398FD38
:050442000FD5F0EA22D5
:10044700C2D5EC30E709B2D5E4C39DFDE49CFCEED0
:1004570030E715B2D5E4C39FFFE49EFE1203F2C353
:10046700E49DFDE49CFC80031203F230D507C3E44E
:060477009FFFE49EFE223F
:0E047D00C3E49FFFE49EFEE49DFDE49CFC2290
:100B2200020CFCE493A3F8E493A34003F68001F2E1
:100B320008DFF48029E493A3F85407240CC8C333D4
:100B4200C4540F4420C8834004F456800146F6DFA3
:100B5200E4800B0102040810204080900F20E47E04
:100B6200019360BCA3FF543F30E509541FFEE49398
:100B7200A360010ECF54C025E060A840B8E493A35F
:100B8200FAE493A3F8E493A3C8C582C8CAC583CA8A
:100B9200F0A3C8C582C8CAC583CADFE9DEE780BE42
:010F350000BB
:00000001FF
